###############################################################################
#
# IAR ELF Linker V8.22.2.15995/W32 for ARM                05/Oct/2019  21:39:55
# Copyright 2007-2018 IAR Systems AB.
#
#    Output file  =  
#        D:\My
#        code\STM\stm32f411e-discovery\broadcaststatemachine\EWARM\broadcaststatemachine\Exe\broadcaststatemachine.out
#    Map file     =  
#        D:\My
#        code\STM\stm32f411e-discovery\broadcaststatemachine\EWARM\broadcaststatemachine\List\broadcaststatemachine.map
#    Command line =  
#        -f C:\Users\Ronald\AppData\Local\Temp\EW606D.tmp ("D:\My
#        code\STM\stm32f411e-discovery\broadcaststatemachine\EWARM\broadcaststatemachine\Obj\BroadcastStateMachine.o"
#        "D:\My
#        code\STM\stm32f411e-discovery\broadcaststatemachine\EWARM\broadcaststatemachine\Obj\Leds.o"
#        "D:\My
#        code\STM\stm32f411e-discovery\broadcaststatemachine\EWARM\broadcaststatemachine\Obj\main.o"
#        "D:\My
#        code\STM\stm32f411e-discovery\broadcaststatemachine\EWARM\broadcaststatemachine\Obj\startup_stm32f407xx.o"
#        "D:\My
#        code\STM\stm32f411e-discovery\broadcaststatemachine\EWARM\broadcaststatemachine\Obj\stm32f4xx_hal.o"
#        "D:\My
#        code\STM\stm32f411e-discovery\broadcaststatemachine\EWARM\broadcaststatemachine\Obj\stm32f4xx_hal_cortex.o"
#        "D:\My
#        code\STM\stm32f411e-discovery\broadcaststatemachine\EWARM\broadcaststatemachine\Obj\stm32f4xx_hal_dma.o"
#        "D:\My
#        code\STM\stm32f411e-discovery\broadcaststatemachine\EWARM\broadcaststatemachine\Obj\stm32f4xx_hal_dma_ex.o"
#        "D:\My
#        code\STM\stm32f411e-discovery\broadcaststatemachine\EWARM\broadcaststatemachine\Obj\stm32f4xx_hal_exti.o"
#        "D:\My
#        code\STM\stm32f411e-discovery\broadcaststatemachine\EWARM\broadcaststatemachine\Obj\stm32f4xx_hal_flash.o"
#        "D:\My
#        code\STM\stm32f411e-discovery\broadcaststatemachine\EWARM\broadcaststatemachine\Obj\stm32f4xx_hal_flash_ex.o"
#        "D:\My
#        code\STM\stm32f411e-discovery\broadcaststatemachine\EWARM\broadcaststatemachine\Obj\stm32f4xx_hal_flash_ramfunc.o"
#        "D:\My
#        code\STM\stm32f411e-discovery\broadcaststatemachine\EWARM\broadcaststatemachine\Obj\stm32f4xx_hal_gpio.o"
#        "D:\My
#        code\STM\stm32f411e-discovery\broadcaststatemachine\EWARM\broadcaststatemachine\Obj\stm32f4xx_hal_msp.o"
#        "D:\My
#        code\STM\stm32f411e-discovery\broadcaststatemachine\EWARM\broadcaststatemachine\Obj\stm32f4xx_hal_pwr.o"
#        "D:\My
#        code\STM\stm32f411e-discovery\broadcaststatemachine\EWARM\broadcaststatemachine\Obj\stm32f4xx_hal_pwr_ex.o"
#        "D:\My
#        code\STM\stm32f411e-discovery\broadcaststatemachine\EWARM\broadcaststatemachine\Obj\stm32f4xx_hal_rcc.o"
#        "D:\My
#        code\STM\stm32f411e-discovery\broadcaststatemachine\EWARM\broadcaststatemachine\Obj\stm32f4xx_hal_rcc_ex.o"
#        "D:\My
#        code\STM\stm32f411e-discovery\broadcaststatemachine\EWARM\broadcaststatemachine\Obj\stm32f4xx_hal_tim.o"
#        "D:\My
#        code\STM\stm32f411e-discovery\broadcaststatemachine\EWARM\broadcaststatemachine\Obj\stm32f4xx_hal_tim_ex.o"
#        "D:\My
#        code\STM\stm32f411e-discovery\broadcaststatemachine\EWARM\broadcaststatemachine\Obj\stm32f4xx_hal_uart.o"
#        "D:\My
#        code\STM\stm32f411e-discovery\broadcaststatemachine\EWARM\broadcaststatemachine\Obj\stm32f4xx_it.o"
#        "D:\My
#        code\STM\stm32f411e-discovery\broadcaststatemachine\EWARM\broadcaststatemachine\Obj\system_stm32f4xx.o"
#        "D:\My
#        code\STM\stm32f411e-discovery\broadcaststatemachine\EWARM\broadcaststatemachine\Obj\TimerModule.o"
#        "D:\My
#        code\STM\stm32f411e-discovery\broadcaststatemachine\EWARM\broadcaststatemachine\Obj\UartProcessing.o"
#        "D:\My
#        code\STM\stm32f411e-discovery\broadcaststatemachine\EWARM\broadcaststatemachine\Obj\UserButton.o"
#        --redirect _Printf=_PrintfFull --redirect _Scanf=_ScanfFull -o "D:\My
#        code\STM\stm32f411e-discovery\broadcaststatemachine\EWARM\broadcaststatemachine\Exe\broadcaststatemachine.out"
#        --map "D:\My
#        code\STM\stm32f411e-discovery\broadcaststatemachine\EWARM\broadcaststatemachine\List\broadcaststatemachine.map"
#        --config "D:\My
#        code\STM\stm32f411e-discovery\broadcaststatemachine\EWARM/stm32f407xx_flash.icf"
#        --semihosting --entry __iar_program_start --vfe --text_out locale)
#
###############################################################################

*******************************************************************************
*** RUNTIME MODEL ATTRIBUTES
***

CppFlavor       = *
__SystemLibrary = DLib
__dlib_version  = 6


*******************************************************************************
*** HEAP SELECTION
***

The basic heap was selected because some modules are built with
size limitations (and not runtime checking), and --advanced_heap
was not specified.


*******************************************************************************
*** PLACEMENT SUMMARY
***

"A0":  place at 0x08000000 { ro section .intvec };
"P1":  place in [from 0x08000000 to 0x080fffff] { ro };
define block CSTACK with size = 1K, alignment = 8 { };
define block HEAP with size = 512, alignment = 8 { };
"P2":  place in [from 0x20000000 to 0x2001ffff] {
          rw, block CSTACK, block HEAP };
initialize by copy { rw };

  Section            Kind        Address    Size  Object
  -------            ----        -------    ----  ------
"A0":                                      0x188
  .intvec            ro code  0x08000000   0x188  startup_stm32f407xx.o [1]
                            - 0x08000188   0x188

"P1":                                     0x246c
  .text              ro code  0x08000188   0x45a  stm32f4xx_hal_uart.o [1]
  .text              ro code  0x080005e4   0x124  stm32f4xx_hal_msp.o [1]
  .text              ro code  0x08000708     0xc  stm32f4xx_hal.o [1]
  .text              ro code  0x08000714   0x350  stm32f4xx_hal_dma.o [1]
  .text              ro code  0x08000a64   0x244  main.o [1]
  .text              ro code  0x08000ca8     0x2  stm32f4xx_hal_uart.o [1]
  .text              ro code  0x08000caa     0x2  stm32f4xx_hal_uart.o [1]
  .text              ro code  0x08000cac   0x1a0  stm32f4xx_hal_rcc.o [1]
  .text              ro code  0x08000e4c    0xc8  stm32f4xx_hal_cortex.o [1]
  .text              ro code  0x08000f14     0x6  ABImemclr4.o [5]
  .text              ro code  0x08000f1c   0x204  stm32f4xx_hal_gpio.o [1]
  .text              ro code  0x08001120    0x34  stm32f4xx_hal.o [1]
  .text              ro code  0x08001154   0x394  stm32f4xx_hal_tim.o [1]
  .text              ro code  0x080014e8    0x3e  stm32f4xx_hal_tim_ex.o [1]
  .text              ro code  0x08001528   0x1b4  TimerModule.o [1]
  .text              ro code  0x080016dc   0x438  BroadcastStateMachine.o [1]
  .text              ro code  0x08001b14   0x2f0  stm32f4xx_hal_rcc.o [1]
  .text              ro code  0x08001e04    0x40  stm32f4xx_hal.o [1]
  .text              ro code  0x08001e44   0x22e  I64DivMod.o [5]
  .text              ro code  0x08002074    0x32  ABImemset48.o [5]
  .text              ro code  0x080020a6     0x2  stm32f4xx_hal_tim.o [1]
  .text              ro code  0x080020a8     0x2  stm32f4xx_hal_tim.o [1]
  .text              ro code  0x080020aa     0x2  stm32f4xx_hal_tim_ex.o [1]
  .text              ro code  0x080020ac     0x2  stm32f4xx_hal_tim.o [1]
  .text              ro code  0x080020ae     0x2  stm32f4xx_hal_tim_ex.o [1]
  .text              ro code  0x080020b0     0x2  stm32f4xx_hal_tim.o [1]
  .text              ro code  0x080020b4   0x124  UserButton.o [1]
  .text              ro code  0x080021d8    0xa8  Leds.o [1]
  .text              ro code  0x08002280     0x2  I64DivZer.o [5]
  .text              ro code  0x08002284    0x60  system_stm32f4xx.o [1]
  Initializer bytes  const    0x080022e4    0x54  <for P2-1>
  .text              ro code  0x08002338    0x40  zero_init3.o [5]
  .text              ro code  0x08002378    0x2c  copy_init3.o [5]
  .text              ro code  0x080023a4    0x28  stm32f4xx_it.o [1]
  .text              ro code  0x080023cc    0x10  stm32f4xx_hal.o [1]
  .text              ro code  0x080023dc    0x28  data_init.o [5]
  .text              ro code  0x08002404    0x22  fpinit_M.o [4]
  .iar.init_table    const    0x08002428    0x24  - Linker created -
  .text              ro code  0x0800244c    0x1e  cmain.o [5]
  .text              ro code  0x0800246a     0x4  low_level_init.o [3]
  .text              ro code  0x0800246e     0x4  exit.o [3]
  .text              ro code  0x08002474     0xa  cexit.o [5]
  .text              ro code  0x08002480    0x14  exit.o [6]
  .text              ro code  0x08002494    0x10  startup_stm32f407xx.o [1]
  .text              ro code  0x080024a4     0xc  cstartup_M.o [5]
  .rodata            const    0x080024b0     0x8  system_stm32f4xx.o [1]
  .text              ro code  0x080024b8     0x4  startup_stm32f407xx.o [1]
  .text              ro code  0x080024bc     0x4  startup_stm32f407xx.o [1]
  .text              ro code  0x080024c0     0x4  startup_stm32f407xx.o [1]
  .text              ro code  0x080024c4     0x4  startup_stm32f407xx.o [1]
  .text              ro code  0x080024c8     0x4  startup_stm32f407xx.o [1]
  .text              ro code  0x080024cc     0x4  startup_stm32f407xx.o [1]
  .text              ro code  0x080024d0     0x4  startup_stm32f407xx.o [1]
  .text              ro code  0x080024d4     0x4  startup_stm32f407xx.o [1]
  .text              ro code  0x080024d8     0x4  startup_stm32f407xx.o [1]
  .text              ro code  0x080024dc     0x4  startup_stm32f407xx.o [1]
  .text              ro code  0x080024e0     0x4  startup_stm32f407xx.o [1]
  .text              ro code  0x080024e4     0x4  startup_stm32f407xx.o [1]
  .text              ro code  0x080024e8     0x4  startup_stm32f407xx.o [1]
  .text              ro code  0x080024ec     0x4  startup_stm32f407xx.o [1]
  .text              ro code  0x080024f0     0x4  startup_stm32f407xx.o [1]
  .text              ro code  0x080024f4     0x4  startup_stm32f407xx.o [1]
  .text              ro code  0x080024f8     0x4  startup_stm32f407xx.o [1]
  .text              ro code  0x080024fc     0x4  startup_stm32f407xx.o [1]
  .text              ro code  0x08002500     0x4  startup_stm32f407xx.o [1]
  .text              ro code  0x08002504     0x4  startup_stm32f407xx.o [1]
  .text              ro code  0x08002508     0x4  startup_stm32f407xx.o [1]
  .text              ro code  0x0800250c     0x4  startup_stm32f407xx.o [1]
  .text              ro code  0x08002510     0x4  startup_stm32f407xx.o [1]
  .text              ro code  0x08002514     0x4  startup_stm32f407xx.o [1]
  .text              ro code  0x08002518     0x4  startup_stm32f407xx.o [1]
  .text              ro code  0x0800251c     0x4  startup_stm32f407xx.o [1]
  .text              ro code  0x08002520     0x4  startup_stm32f407xx.o [1]
  .text              ro code  0x08002524     0x4  startup_stm32f407xx.o [1]
  .text              ro code  0x08002528     0x4  startup_stm32f407xx.o [1]
  .text              ro code  0x0800252c     0x4  startup_stm32f407xx.o [1]
  .text              ro code  0x08002530     0x4  startup_stm32f407xx.o [1]
  .text              ro code  0x08002534     0x4  startup_stm32f407xx.o [1]
  .text              ro code  0x08002538     0x4  startup_stm32f407xx.o [1]
  .text              ro code  0x0800253c     0x4  startup_stm32f407xx.o [1]
  .text              ro code  0x08002540     0x4  startup_stm32f407xx.o [1]
  .text              ro code  0x08002544     0x4  startup_stm32f407xx.o [1]
  .text              ro code  0x08002548     0x4  startup_stm32f407xx.o [1]
  .text              ro code  0x0800254c     0x4  startup_stm32f407xx.o [1]
  .text              ro code  0x08002550     0x4  startup_stm32f407xx.o [1]
  .text              ro code  0x08002554     0x4  startup_stm32f407xx.o [1]
  .text              ro code  0x08002558     0x4  startup_stm32f407xx.o [1]
  .text              ro code  0x0800255c     0x4  startup_stm32f407xx.o [1]
  .text              ro code  0x08002560     0x4  startup_stm32f407xx.o [1]
  .text              ro code  0x08002564     0x4  startup_stm32f407xx.o [1]
  .text              ro code  0x08002568     0x4  startup_stm32f407xx.o [1]
  .text              ro code  0x0800256c     0x4  startup_stm32f407xx.o [1]
  .text              ro code  0x08002570     0x4  startup_stm32f407xx.o [1]
  .text              ro code  0x08002574     0x4  startup_stm32f407xx.o [1]
  .text              ro code  0x08002578     0x4  startup_stm32f407xx.o [1]
  .text              ro code  0x0800257c     0x4  startup_stm32f407xx.o [1]
  .text              ro code  0x08002580     0x4  startup_stm32f407xx.o [1]
  .text              ro code  0x08002584     0x4  startup_stm32f407xx.o [1]
  .text              ro code  0x08002588     0x4  startup_stm32f407xx.o [1]
  .text              ro code  0x0800258c     0x4  startup_stm32f407xx.o [1]
  .text              ro code  0x08002590     0x4  startup_stm32f407xx.o [1]
  .text              ro code  0x08002594     0x4  startup_stm32f407xx.o [1]
  .text              ro code  0x08002598     0x4  startup_stm32f407xx.o [1]
  .text              ro code  0x0800259c     0x4  startup_stm32f407xx.o [1]
  .text              ro code  0x080025a0     0x4  startup_stm32f407xx.o [1]
  .text              ro code  0x080025a4     0x4  startup_stm32f407xx.o [1]
  .text              ro code  0x080025a8     0x4  startup_stm32f407xx.o [1]
  .text              ro code  0x080025ac     0x4  startup_stm32f407xx.o [1]
  .text              ro code  0x080025b0     0x4  startup_stm32f407xx.o [1]
  .text              ro code  0x080025b4     0x4  startup_stm32f407xx.o [1]
  .text              ro code  0x080025b8     0x4  startup_stm32f407xx.o [1]
  .text              ro code  0x080025bc     0x4  startup_stm32f407xx.o [1]
  .text              ro code  0x080025c0     0x4  startup_stm32f407xx.o [1]
  .text              ro code  0x080025c4     0x4  startup_stm32f407xx.o [1]
  .text              ro code  0x080025c8     0x4  startup_stm32f407xx.o [1]
  .text              ro code  0x080025cc     0x4  startup_stm32f407xx.o [1]
  .text              ro code  0x080025d0     0x4  startup_stm32f407xx.o [1]
  .text              ro code  0x080025d4     0x4  startup_stm32f407xx.o [1]
  .text              ro code  0x080025d8     0x4  startup_stm32f407xx.o [1]
  .text              ro code  0x080025dc     0x4  startup_stm32f407xx.o [1]
  .text              ro code  0x080025e0     0x4  startup_stm32f407xx.o [1]
  .text              ro code  0x080025e4     0x4  startup_stm32f407xx.o [1]
  .text              ro code  0x080025e8     0x4  startup_stm32f407xx.o [1]
  .text              ro code  0x080025ec     0x4  startup_stm32f407xx.o [1]
  .text              ro code  0x080025f0     0x4  startup_stm32f407xx.o [1]
  .rodata            const    0x080025f4     0x0  zero_init3.o [5]
  .rodata            const    0x080025f4     0x0  copy_init3.o [5]
                            - 0x080025f4  0x246c

"P2", part 1 of 3:                          0x54
  P2-1                        0x20000000    0x54  <Init block>
    .data            inited   0x20000000    0x20  BroadcastStateMachine.o [1]
    .data            inited   0x20000020    0x20  BroadcastStateMachine.o [1]
    .data            inited   0x20000040     0xc  stm32f4xx_hal.o [1]
    .data            inited   0x2000004c     0x4  system_stm32f4xx.o [1]
    .data            inited   0x20000050     0x4  Leds.o [1]
                            - 0x20000054    0x54

"P2", part 2 of 3:                         0x218
  .bss               zero     0x20000054   0x100  TimerModule.o [1]
  .bss               zero     0x20000154    0x84  main.o [1]
  .bss               zero     0x200001d8    0x60  main.o [1]
  .bss               zero     0x20000238    0x24  BroadcastStateMachine.o [1]
  .bss               zero     0x2000025c     0x8  UserButton.o [1]
  .bss               zero     0x20000264     0x4  TimerModule.o [1]
  .bss               zero     0x20000268     0x1  UartProcessing.o [1]
                            - 0x20000269   0x215

"P2", part 3 of 3:                         0x400
  CSTACK                      0x20000270   0x400  <Block>
    CSTACK           uninit   0x20000270   0x400  <Block tail>
                            - 0x20000670   0x400


*******************************************************************************
*** INIT TABLE
***

          Address     Size
          -------     ----
Zero (__iar_zero_init3)
    1 destination range, total size 0x215:
          0x20000054  0x215

Copy (__iar_copy_init3)
    1 source range, total size 0x54:
          0x080022e4   0x54
    1 destination range, total size 0x54:
          0x20000000   0x54



*******************************************************************************
*** MODULE SUMMARY
***

    Module                   ro code  ro data  rw data
    ------                   -------  -------  -------
D:\My code\STM\stm32f411e-discovery\broadcaststatemachine\EWARM\broadcaststatemachine\Obj: [1]
    BroadcastStateMachine.o    1 080       64      100
    Leds.o                       168        4        4
    TimerModule.o                436               260
    UartProcessing.o                                 1
    UserButton.o                 292                 8
    main.o                       580               228
    startup_stm32f407xx.o        724
    stm32f4xx_hal.o              144       12       12
    stm32f4xx_hal_cortex.o       200
    stm32f4xx_hal_dma.o          848
    stm32f4xx_hal_gpio.o         516
    stm32f4xx_hal_msp.o          292
    stm32f4xx_hal_rcc.o        1 168
    stm32f4xx_hal_tim.o          924
    stm32f4xx_hal_tim_ex.o        66
    stm32f4xx_hal_uart.o       1 118
    stm32f4xx_it.o                40
    system_stm32f4xx.o            96       12        4
    --------------------------------------------------
    Total:                     8 692       92      617

command line: [2]
    --------------------------------------------------
    Total:

dl7M_tln.a: [3]
    exit.o                         4
    low_level_init.o               4
    --------------------------------------------------
    Total:                         8

m7M_tls.a: [4]
    fpinit_M.o                    34
    --------------------------------------------------
    Total:                        34

rt7M_tl.a: [5]
    ABImemclr4.o                   6
    ABImemset48.o                 50
    I64DivMod.o                  558
    I64DivZer.o                    2
    cexit.o                       10
    cmain.o                       30
    copy_init3.o                  44
    cstartup_M.o                  12
    data_init.o                   40
    zero_init3.o                  64
    --------------------------------------------------
    Total:                       816

shb_l.a: [6]
    exit.o                        20
    --------------------------------------------------
    Total:                        20

    Gaps                          16        2
    Linker created                         36    1 024
------------------------------------------------------
    Grand Total:               9 586      130    1 641


*******************************************************************************
*** ENTRY LIST
***

Entry                      Address   Size  Type      Object
-----                      -------   ----  ----      ------
.iar.init_table$$Base   0x08002428          --   Gb  - Linker created -
.iar.init_table$$Limit  0x0800244c          --   Gb  - Linker created -
?main                   0x0800244d         Code  Gb  cmain.o [5]
AHBPrescTable           0x080022d4   0x10  Data  Gb  system_stm32f4xx.o [1]
APBPrescTable           0x080024b0    0x8  Data  Gb  system_stm32f4xx.o [1]
BusFault_Handler        0x080023ab    0x2  Code  Gb  stm32f4xx_it.o [1]
CSTACK$$Base            0x20000270          --   Gb  - Linker created -
CSTACK$$Limit           0x20000670          --   Gb  - Linker created -
DMA1_Stream5_IRQHandler
                        0x080023b9    0x6  Code  Gb  stm32f4xx_it.o [1]
DMA_CalcBaseAndBitshift
                        0x08000a35   0x28  Code  Lc  stm32f4xx_hal_dma.o [1]
DMA_CalcBaseAndBitshift::flagBitshiftOffset
                        0x08000a5c    0x8  Data  Lc  stm32f4xx_hal_dma.o [1]
DMA_SetConfig           0x08000a15   0x20  Code  Lc  stm32f4xx_hal_dma.o [1]
DebugMon_Handler        0x080023b1    0x2  Code  Gb  stm32f4xx_it.o [1]
Error_Handler           0x08000c89    0x2  Code  Gb  main.o [1]
HAL_DMA_IRQHandler      0x08000865  0x188  Code  Gb  stm32f4xx_hal_dma.o [1]
HAL_DMA_Init            0x08000715   0xe6  Code  Gb  stm32f4xx_hal_dma.o [1]
HAL_DMA_Start_IT        0x080007fb   0x6a  Code  Gb  stm32f4xx_hal_dma.o [1]
HAL_GPIO_Init           0x08000f1d  0x1b2  Code  Gb  stm32f4xx_hal_gpio.o [1]
HAL_GPIO_ReadPin        0x080010cf    0xc  Code  Gb  stm32f4xx_hal_gpio.o [1]
HAL_GPIO_TogglePin      0x080010e3    0xc  Code  Gb  stm32f4xx_hal_gpio.o [1]
HAL_GPIO_WritePin       0x080010db    0x8  Code  Gb  stm32f4xx_hal_gpio.o [1]
HAL_GetTick             0x08000709    0xc  Code  Wk  stm32f4xx_hal.o [1]
HAL_IncTick             0x080023cd   0x10  Code  Wk  stm32f4xx_hal.o [1]
HAL_Init                0x08001121   0x30  Code  Gb  stm32f4xx_hal.o [1]
HAL_InitTick            0x08001e05   0x40  Code  Wk  stm32f4xx_hal.o [1]
HAL_MspInit             0x080005e5   0x38  Code  Gb  stm32f4xx_hal_msp.o [1]
HAL_NVIC_EnableIRQ      0x08000ebf   0x16  Code  Gb  stm32f4xx_hal_cortex.o [1]
HAL_NVIC_SetPriority    0x08000e85   0x3a  Code  Gb  stm32f4xx_hal_cortex.o [1]
HAL_NVIC_SetPriorityGrouping
                        0x08000e6b   0x1a  Code  Gb  stm32f4xx_hal_cortex.o [1]
HAL_RCC_ClockConfig     0x08000cad   0xfe  Code  Gb  stm32f4xx_hal_rcc.o [1]
HAL_RCC_GetPCLK1Freq    0x08000db7   0x10  Code  Gb  stm32f4xx_hal_rcc.o [1]
HAL_RCC_GetPCLK2Freq    0x08000dc7    0xe  Code  Gb  stm32f4xx_hal_rcc.o [1]
HAL_RCC_OscConfig       0x08001b15  0x2f0  Code  Wk  stm32f4xx_hal_rcc.o [1]
HAL_SYSTICK_Config      0x08000ed5   0x28  Code  Gb  stm32f4xx_hal_cortex.o [1]
HAL_TIMEx_BreakCallback
                        0x080020ab    0x2  Code  Wk  stm32f4xx_hal_tim_ex.o [1]
HAL_TIMEx_CommutCallback
                        0x080020af    0x2  Code  Wk  stm32f4xx_hal_tim_ex.o [1]
HAL_TIMEx_MasterConfigSynchronization
                        0x080014e9   0x3e  Code  Gb  stm32f4xx_hal_tim_ex.o [1]
HAL_TIM_Base_Init       0x08001155   0x1a  Code  Gb  stm32f4xx_hal_tim.o [1]
HAL_TIM_Base_MspInit    0x0800061d   0x30  Code  Gb  stm32f4xx_hal_msp.o [1]
HAL_TIM_Base_Start_IT   0x0800116f   0x20  Code  Gb  stm32f4xx_hal_tim.o [1]
HAL_TIM_ConfigClockSource
                        0x080012fb   0x90  Code  Gb  stm32f4xx_hal_tim.o [1]
HAL_TIM_IRQHandler      0x080011b3  0x142  Code  Gb  stm32f4xx_hal_tim.o [1]
HAL_TIM_PeriodElapsedCallback
                        0x08000c4b    0x4  Code  Gb  main.o [1]
HAL_UART_Init           0x08000189   0x1e  Code  Gb  stm32f4xx_hal_uart.o [1]
HAL_UART_MspInit        0x0800064d   0x98  Code  Gb  stm32f4xx_hal_msp.o [1]
HAL_UART_Receive_DMA    0x080002b3   0x92  Code  Gb  stm32f4xx_hal_uart.o [1]
HAL_UART_RxCpltCallback
                        0x08000c4f   0x12  Code  Gb  main.o [1]
HAL_UART_Transmit       0x08000201   0xaa  Code  Gb  stm32f4xx_hal_uart.o [1]
HardFault_Handler       0x080023a7    0x2  Code  Gb  stm32f4xx_it.o [1]
LedBlueFunction         0x08002221    0x4  Code  Gb  Leds.o [1]
LedBlueTurnOff          0x08002253    0x8  Code  Gb  Leds.o [1]
LedBlueTurnOn           0x0800224b    0x8  Code  Gb  Leds.o [1]
LedGetBlueTimerId       0x08002271    0x6  Code  Gb  Leds.o [1]
LedGetRedTimerId        0x0800226b    0x6  Code  Gb  Leds.o [1]
LedGreenFunction        0x0800222d    0x6  Code  Gb  Leds.o [1]
LedGreenTurnOn          0x0800225b    0x8  Code  Gb  Leds.o [1]
LedInit                 0x080021d9   0x36  Code  Gb  Leds.o [1]
LedOrangeFunction       0x08002235    0x6  Code  Gb  Leds.o [1]
LedOrangeTurnOn         0x08002263    0x8  Code  Gb  Leds.o [1]
LedRedFunction          0x08002219    0x6  Code  Gb  Leds.o [1]
LedRedTurnOff           0x0800223f    0x2  Code  Gb  Leds.o [1]
LedRedTurnOn            0x0800223b    0x4  Code  Gb  Leds.o [1]
MemManage_Handler       0x080023a9    0x2  Code  Gb  stm32f4xx_it.o [1]
NMI_Handler             0x080023a5    0x2  Code  Gb  stm32f4xx_it.o [1]
PendSV_Handler          0x080023b3    0x2  Code  Gb  stm32f4xx_it.o [1]
Region$$Table$$Base     0x08002428          --   Gb  - Linker created -
Region$$Table$$Limit    0x0800244c          --   Gb  - Linker created -
SM_CommonTasks          0x08001733    0x4  Code  Gb  BroadcastStateMachine.o [1]
SM_Init                 0x080016dd   0x56  Code  Gb  BroadcastStateMachine.o [1]
SM_State1Machine1       0x08001739   0x28  Code  Gb  BroadcastStateMachine.o [1]
SM_State1Machine2       0x0800180b   0x1c  Code  Gb  BroadcastStateMachine.o [1]
SM_State1Machine3       0x080018a9    0x2  Code  Gb  BroadcastStateMachine.o [1]
SM_State2Machine1       0x08001761   0x38  Code  Gb  BroadcastStateMachine.o [1]
SM_State2Machine2       0x0800183b   0x1e  Code  Gb  BroadcastStateMachine.o [1]
SM_State3Machine1       0x08001799   0x36  Code  Gb  BroadcastStateMachine.o [1]
SM_State3Machine2       0x08001859   0x1e  Code  Gb  BroadcastStateMachine.o [1]
SM_State4Machine1       0x080017d7   0x34  Code  Gb  BroadcastStateMachine.o [1]
SM_State4Machine2       0x08001877   0x28  Code  Gb  BroadcastStateMachine.o [1]
SM_StateMachineBlue     0x20000240    0x8  Data  Gb  BroadcastStateMachine.o [1]
SM_StateMachineGreen    0x20000248    0x8  Data  Gb  BroadcastStateMachine.o [1]
SM_StateMachineOrange   0x20000250    0x8  Data  Gb  BroadcastStateMachine.o [1]
SM_StateMachineRed      0x20000238    0x8  Data  Gb  BroadcastStateMachine.o [1]
SVC_Handler             0x080023af    0x2  Code  Gb  stm32f4xx_it.o [1]
SysTick_Handler         0x080023b5    0x4  Code  Gb  stm32f4xx_it.o [1]
SystemClock_Config      0x08000bbb   0x90  Code  Gb  main.o [1]
SystemCoreClock         0x2000004c    0x4  Data  Gb  system_stm32f4xx.o [1]
SystemInit              0x08002285   0x3a  Code  Gb  system_stm32f4xx.o [1]
TIM2_IRQHandler         0x080023bf    0x6  Code  Gb  stm32f4xx_it.o [1]
TIM_Base_SetConfig      0x080013b5   0x96  Code  Gb  stm32f4xx_hal_tim.o [1]
TIM_ETR_SetConfig       0x080014cf   0x14  Code  Gb  stm32f4xx_hal_tim.o [1]
TIM_ITRx_SetConfig      0x080014bf   0x10  Code  Lc  stm32f4xx_hal_tim.o [1]
TIM_TI1_ConfigInputStage
                        0x0800147d   0x1e  Code  Lc  stm32f4xx_hal_tim.o [1]
TIM_TI2_ConfigInputStage
                        0x0800149b   0x24  Code  Lc  stm32f4xx_hal_tim.o [1]
TmrChangeTimerValue     0x0800165f   0x24  Code  Gb  TimerModule.o [1]
TmrCreate               0x08001553   0x1a  Code  Gb  TimerModule.o [1]
TmrCreateTimer          0x0800162b   0x34  Code  Gb  TimerModule.o [1]
TmrDelete               0x080015db    0x2  Code  Gb  TimerModule.o [1]
TmrInit                 0x08001529   0x2a  Code  Gb  TimerModule.o [1]
TmrPopulate             0x0800156d   0x2a  Code  Gb  TimerModule.o [1]
TmrProcessTimerArray    0x080015dd   0x4e  Code  Gb  TimerModule.o [1]
TmrReset                0x080015b9   0x22  Code  Gb  TimerModule.o [1]
TmrStart                0x08001597   0x20  Code  Gb  TimerModule.o [1]
TmrStop                 0x080015b7    0x2  Code  Gb  TimerModule.o [1]
UART_DMAError           0x08000385   0x4a  Code  Lc  stm32f4xx_hal_uart.o [1]
UART_DMAReceiveCplt     0x08000345   0x38  Code  Lc  stm32f4xx_hal_uart.o [1]
UART_DMARxHalfCplt      0x0800037d    0x6  Code  Lc  stm32f4xx_hal_uart.o [1]
UART_EndRxTransfer      0x08000445   0x1c  Code  Lc  stm32f4xx_hal_uart.o [1]
UART_EndTxTransfer      0x08000433   0x12  Code  Lc  stm32f4xx_hal_uart.o [1]
UART_SetConfig          0x08000461  0x13a  Code  Lc  stm32f4xx_hal_uart.o [1]
UART_WaitOnFlagUntilTimeout
                        0x080003cf   0x56  Code  Lc  stm32f4xx_hal_uart.o [1]
UsageFault_Handler      0x080023ad    0x2  Code  Gb  stm32f4xx_it.o [1]
UserButtonCheck         0x080020ff   0x32  Code  Gb  UserButton.o [1]
UserButtonDbnCheck      0x08002131   0x1e  Code  Gb  UserButton.o [1]
UserButtonDelayEnable   0x08002177   0x2e  Code  Gb  UserButton.o [1]
UserButtonDelayExp      0x080021a5    0x8  Code  Gb  UserButton.o [1]
UserButtonGetDbn        0x08002169    0xe  Code  Gb  UserButton.o [1]
UserButtonGetPressed    0x08002155    0xe  Code  Gb  UserButton.o [1]
UserButtonInit          0x080020b5   0x4a  Code  Gb  UserButton.o [1]
UserButtonIsDelayed     0x080021ad    0x6  Code  Gb  UserButton.o [1]
UserButtonSetDbn        0x08002163    0x6  Code  Gb  UserButton.o [1]
UserButtonSetPressed    0x0800214f    0x6  Code  Gb  UserButton.o [1]
UserButtonStartDelay    0x080021b3   0x1c  Code  Gb  UserButton.o [1]
__NVIC_SetPriority      0x08000e4d   0x1e  Code  Lc  stm32f4xx_hal_cortex.o [1]
__aeabi_ldiv0           0x08002281         Code  Gb  I64DivZer.o [5]
__aeabi_memclr4         0x08000f15         Code  Gb  ABImemclr4.o [5]
__aeabi_uldivmod        0x08001e45         Code  Gb  I64DivMod.o [5]
__cmain                 0x0800244d         Code  Gb  cmain.o [5]
__exit                  0x08002481   0x14  Code  Gb  exit.o [6]
__iar_Memset4_word      0x08002075         Code  Gb  ABImemset48.o [5]
__iar_Memset8_word      0x08002075         Code  Gb  ABImemset48.o [5]
__iar_copy_init3        0x08002379   0x2c  Code  Gb  copy_init3.o [5]
__iar_data_init3        0x080023dd   0x28  Code  Gb  data_init.o [5]
__iar_init_vfp          0x08002405         Code  Gb  fpinit_M.o [4]
__iar_program_start     0x080024a5         Code  Gb  cstartup_M.o [5]
__iar_systems$$module {Abs}
                        0x00000001         Data  Gb  command line/config [2]
__iar_zero_init3        0x08002339   0x40  Code  Gb  zero_init3.o [5]
__low_level_init        0x0800246b    0x4  Code  Gb  low_level_init.o [3]
__vector_table          0x08000000         Data  Gb  startup_stm32f407xx.o [1]
_call_main              0x08002459         Code  Gb  cmain.o [5]
_exit                   0x08002475         Code  Gb  cexit.o [5]
_main                   0x08002467         Code  Gb  cmain.o [5]
broadcastUartValue      0x20000268    0x1  Data  Gb  UartProcessing.o [1]
exit                    0x0800246f    0x4  Code  Gb  exit.o [3]
hdma_usart2_rx          0x200001d8   0x60  Data  Gb  main.o [1]
htim2                   0x20000198   0x40  Data  Gb  main.o [1]
huart2                  0x20000158   0x40  Data  Gb  main.o [1]
m_DeleteTimer           0x080016a5   0x2e  Code  Gb  TimerModule.o [1]
m_Htim                  0x20000264    0x4  Data  Lc  TimerModule.o [1]
m_StopTimer             0x08001683   0x22  Code  Gb  TimerModule.o [1]
m_TmrModuleArray        0x20000054  0x100  Data  Lc  TimerModule.o [1]
m_gotoBlueState1        0x08001a25   0x20  Code  Lc  BroadcastStateMachine.o [1]
m_gotoRedState1         0x08001a01   0x24  Code  Lc  BroadcastStateMachine.o [1]
m_huart                 0x20000258    0x4  Data  Lc  BroadcastStateMachine.o [1]
m_machine1State1Event1  0x080018ad   0x2c  Code  Lc  BroadcastStateMachine.o [1]
m_machine1State1Event2  0x080018d9    0x2  Code  Lc  BroadcastStateMachine.o [1]
m_machine1State2Event1  0x080018dd   0x2c  Code  Lc  BroadcastStateMachine.o [1]
m_machine1State2Event2  0x08001913    0x2  Code  Lc  BroadcastStateMachine.o [1]
m_machine1State3Event1  0x08001915   0x30  Code  Lc  BroadcastStateMachine.o [1]
m_machine1State3Event2  0x08001945    0x2  Code  Lc  BroadcastStateMachine.o [1]
m_machine1State4Event1  0x08001947    0x2  Code  Lc  BroadcastStateMachine.o [1]
m_machine1State4Event2  0x08001949    0x2  Code  Lc  BroadcastStateMachine.o [1]
m_machine2State1Event1  0x0800194d   0x2c  Code  Lc  BroadcastStateMachine.o [1]
m_machine2State1Event2  0x08001985    0x2  Code  Lc  BroadcastStateMachine.o [1]
m_machine2State2Event1  0x08001989   0x2c  Code  Lc  BroadcastStateMachine.o [1]
m_machine2State2Event2  0x080019bf    0x2  Code  Lc  BroadcastStateMachine.o [1]
m_machine2State3Event1  0x080019c1   0x30  Code  Lc  BroadcastStateMachine.o [1]
m_machine2State3Event2  0x080019fb    0x2  Code  Lc  BroadcastStateMachine.o [1]
m_machine2State4Event1  0x080019fd    0x2  Code  Lc  BroadcastStateMachine.o [1]
m_machine2State4Event2  0x080019ff    0x2  Code  Lc  BroadcastStateMachine.o [1]
m_rxData                0x20000154    0x1  Data  Lc  main.o [1]
m_tmrBlueBlinkingId     0x20000051    0x1  Data  Lc  Leds.o [1]
m_tmrBtnDebounceId      0x2000025e    0x1  Data  Lc  UserButton.o [1]
m_tmrGreenBlinkingId    0x20000052    0x1  Data  Lc  Leds.o [1]
m_tmrOrangeBlinkingId   0x20000053    0x1  Data  Lc  Leds.o [1]
m_tmrRedBlinkingId      0x20000050    0x1  Data  Lc  Leds.o [1]
m_usrButtonDebounce     0x2000025d    0x1  Data  Lc  UserButton.o [1]
m_usrButtonDelay        0x20000260    0x1  Data  Lc  UserButton.o [1]
m_usrButtonDelayId      0x20000261    0x1  Data  Lc  UserButton.o [1]
m_usrButtonDelayValue   0x20000262    0x2  Data  Lc  UserButton.o [1]
m_usrButtonPressed      0x2000025c    0x1  Data  Lc  UserButton.o [1]
m_usrDelayEnable        0x2000025f    0x1  Data  Lc  UserButton.o [1]
main                    0x08000a65  0x156  Code  Gb  main.o [1]
stateEventTableMachine1
                        0x20000000   0x20  Data  Gb  BroadcastStateMachine.o [1]
stateEventTableMachine2
                        0x20000020   0x20  Data  Gb  BroadcastStateMachine.o [1]
uwTick                  0x20000044    0x4  Data  Gb  stm32f4xx_hal.o [1]
uwTickFreq              0x20000040    0x1  Data  Gb  stm32f4xx_hal.o [1]
uwTickPrio              0x20000048    0x4  Data  Gb  stm32f4xx_hal.o [1]


[1] = D:\My code\STM\stm32f411e-discovery\broadcaststatemachine\EWARM\broadcaststatemachine\Obj
[2] = command line
[3] = dl7M_tln.a
[4] = m7M_tls.a
[5] = rt7M_tl.a
[6] = shb_l.a

  9 586 bytes of readonly  code memory
    130 bytes of readonly  data memory
  1 641 bytes of readwrite data memory

Errors: none
Warnings: none
